BL51 BANKED LINKER/LOCATER V6.22.2.0                                                    05/05/2022  21:30:59  PAGE 1


BL51 BANKED LINKER/LOCATER V6.22.2.0, INVOKED BY:
C:\KEIL_V5\C51\BIN\BL51.EXE .\Objects\main.obj, .\Objects\delay.obj, .\Objects\display.obj TO .\Objects\MCU_1 PRINT (.\L
>> istings\MCU_1.m51)


MEMORY MODEL: LARGE


INPUT MODULES INCLUDED:
  .\Objects\main.obj (MAIN)
  .\Objects\delay.obj (DELAY)
  .\Objects\display.obj (DISPLAY)
  C:\KEIL_V5\C51\LIB\C51L.LIB (?C_STARTUP)
  C:\KEIL_V5\C51\LIB\C51L.LIB (?C_INIT)


LINK MAP OF MODULE:  .\Objects\MCU_1 (MAIN)


            TYPE    BASE      LENGTH    RELOCATION   SEGMENT NAME
            -----------------------------------------------------

            * * * * * * *   D A T A   M E M O R Y   * * * * * * *
            REG     0000H     0008H     ABSOLUTE     "REG BANK 0"
            IDATA   0008H     0001H     UNIT         ?STACK

            * * * * * * *  X D A T A   M E M O R Y  * * * * * * *
            XDATA   0000H     0060H     UNIT         ?XD?DISPLAY
            XDATA   0060H     0004H     UNIT         ?XD?TEST?DISPLAY
            XDATA   0064H     0004H     UNIT         _XDATA_GROUP_
            XDATA   0068H     0002H     UNIT         ?XD?MAIN

            * * * * * * *   C O D E   M E M O R Y   * * * * * * *
            CODE    0000H     0003H     ABSOLUTE     
            CODE    0003H     0104H     UNIT         ?PR?_NAME?DISPLAY
            CODE    0107H     00D7H     UNIT         ?PR?CLEAR?DISPLAY
            CODE    01DEH     00D7H     UNIT         ?PR?MINICLEAR?DISPLAY
            CODE    02B5H     00D7H     UNIT         ?PR?TEST?DISPLAY
            CODE    038CH     008CH     UNIT         ?C_C51STARTUP
            CODE    0418H     006EH     UNIT         ?C_INITSEG
            CODE    0486H     0034H     UNIT         ?PR?WRITE?DISPLAY
            CODE    04BAH     0024H     UNIT         ?PR?MAIN?MAIN
            CODE    04DEH     0020H     UNIT         ?PR?_DELAY?DELAY
            CODE    04FEH     001CH     UNIT         ?PR?INIT?DISPLAY
            CODE    051AH     000BH     UNIT         ?PR?DELAY100US?DELAY
            CODE    0525H     0007H     UNIT         ?PR?_WRITEDATA?DISPLAY
            CODE    052CH     0007H     UNIT         ?PR?_SETCOMMAND?DISPLAY
            CODE    0533H     0007H     UNIT         ?PR?_SETPAGE?DISPLAY
            CODE    053AH     0007H     UNIT         ?PR?_SETLINE?DISPLAY
            CODE    0541H     0007H     UNIT         ?PR?_SETY?DISPLAY



OVERLAY MAP OF MODULE:   .\Objects\MCU_1 (MAIN)


SEGMENT                           XDATA_GROUP
  +--> CALLED SEGMENT           START    LENGTH
BL51 BANKED LINKER/LOCATER V6.22.2.0                                                  05/05/2022  21:30:59  PAGE 2


-----------------------------------------------
?C_C51STARTUP                   -----    -----
  +--> ?PR?MAIN?MAIN
  +--> ?C_INITSEG

?PR?MAIN?MAIN                   -----    -----
  +--> ?PR?INIT?DISPLAY
  +--> ?PR?CLEAR?DISPLAY
  +--> ?PR?_NAME?DISPLAY
  +--> ?PR?MINICLEAR?DISPLAY

?PR?INIT?DISPLAY                -----    -----
  +--> ?PR?WRITE?DISPLAY

?PR?WRITE?DISPLAY               -----    -----
  +--> ?PR?_DELAY?DELAY

?PR?CLEAR?DISPLAY               0064H    0004H
  +--> ?PR?WRITE?DISPLAY

?PR?_NAME?DISPLAY               0064H    0003H
  +--> ?PR?WRITE?DISPLAY

?PR?MINICLEAR?DISPLAY           0064H    0004H
  +--> ?PR?WRITE?DISPLAY



SYMBOL TABLE OF MODULE:  .\Objects\MCU_1 (MAIN)

  VALUE           TYPE          NAME
  ----------------------------------

  -------         MODULE        MAIN
  C:0000H         SYMBOL        _ICE_DUMMY_
  D:0090H         PUBLIC        P1
  D:00B0H         PUBLIC        P3
  D:00A8H         PUBLIC        IE
  D:00B8H         PUBLIC        IP
  C:04BAH         PUBLIC        main
  X:0068H         PUBLIC        line
  D:0098H         PUBLIC        SCON
  D:0088H         PUBLIC        TCON
  D:00C8H         PUBLIC        T2CON
  D:00D0H         PUBLIC        PSW
  -------         PROC          MAIN
  C:04BAH         LINE#         13
  C:04BAH         LINE#         14
  C:04BAH         LINE#         15
  C:04BDH         LINE#         16
  C:04C0H         LINE#         18
  C:04C0H         LINE#         19
  C:04C0H         LINE#         21
  C:04CBH         LINE#         22
  C:04CEH         LINE#         23
  C:04DCH         LINE#         25
  -------         ENDPROC       MAIN
BL51 BANKED LINKER/LOCATER V6.22.2.0                                                  05/05/2022  21:30:59  PAGE 3


  -------         ENDMOD        MAIN

  -------         MODULE        DELAY
  C:0000H         SYMBOL        _ICE_DUMMY_
  C:051AH         PUBLIC        delay100us
  C:04DEH         PUBLIC        _delay
  -------         PROC          DELAY100US
  -------         DO            
  D:0007H         SYMBOL        i
  D:0006H         SYMBOL        j
  -------         ENDDO         
  C:051AH         LINE#         3
  C:051AH         LINE#         4
  C:051AH         LINE#         7
  C:051BH         LINE#         8
  C:051CH         LINE#         9
  C:051EH         LINE#         10
  C:0520H         LINE#         12
  C:0520H         LINE#         13
  C:0522H         LINE#         14
  C:0524H         LINE#         15
  -------         ENDPROC       DELAY100US
  -------         PROC          _DELAY
  D:0006H         SYMBOL        n
  -------         DO            
  D:0006H         SYMBOL        i
  D:0004H         SYMBOL        j
  -------         ENDDO         
  C:04DEH         LINE#         24
  C:04DEH         LINE#         26
  C:04DEH         LINE#         27
  C:04E9H         LINE#         28
  C:04FDH         LINE#         29
  -------         ENDPROC       _DELAY
  -------         ENDMOD        DELAY

  -------         MODULE        DISPLAY
  C:0000H         SYMBOL        _ICE_DUMMY_
  D:0090H         PUBLIC        P1
  D:00B0H         PUBLIC        P3
  C:0107H         PUBLIC        clear
  X:0000H         PUBLIC        Z2
  D:00A8H         PUBLIC        IE
  C:052CH         PUBLIC        _setCommand
  D:00B8H         PUBLIC        IP
  C:0003H         PUBLIC        _name
  B:00B0H.0       PUBLIC        RS
  C:0541H         PUBLIC        _setY
  B:00B0H.1       PUBLIC        RW
  C:0525H         PUBLIC        _writeData
  C:04AAH         PUBLIC        write
  D:0098H         PUBLIC        SCON
  D:0088H         PUBLIC        TCON
  C:04FEH         PUBLIC        init
  C:01DEH         PUBLIC        miniclear
  C:02B5H         PUBLIC        test
  B:00B0H.2       PUBLIC        E
BL51 BANKED LINKER/LOCATER V6.22.2.0                                                  05/05/2022  21:30:59  PAGE 4


  C:0533H         PUBLIC        _setPage
  B:00B0H.4       PUBLIC        CSA
  B:00B0H.5       PUBLIC        CSB
  C:053AH         PUBLIC        _setLine
  X:0030H         PUBLIC        Z
  D:00C8H         PUBLIC        T2CON
  D:00D0H         PUBLIC        PSW
  C:0486H         SYMBOL        L?0071
  C:04A4H         SYMBOL        L?0072
  -------         PROC          L?0070
  -------         ENDPROC       L?0070
  C:0486H         SYMBOL        L?0071
  C:04A4H         SYMBOL        L?0072
  -------         PROC          WRITE
  C:04AAH         LINE#         30
  C:04AAH         LINE#         31
  C:04AAH         LINE#         32
  C:04ACH         LINE#         33
  C:04AEH         LINE#         34
  C:04B0H         LINE#         35
  C:04B7H         LINE#         36
  C:04B9H         LINE#         37
  -------         ENDPROC       WRITE
  -------         PROC          _WRITEDATA
  D:0007H         SYMBOL        d
  C:0525H         LINE#         39
  C:0525H         LINE#         40
  C:0525H         LINE#         41
  C:0527H         LINE#         42
  C:0529H         LINE#         43
  C:052BH         LINE#         44
  -------         ENDPROC       _WRITEDATA
  -------         PROC          _SETCOMMAND
  D:0007H         SYMBOL        d
  C:052CH         LINE#         46
  C:052CH         LINE#         47
  C:052CH         LINE#         48
  C:052EH         LINE#         49
  C:0530H         LINE#         50
  C:0532H         LINE#         51
  -------         ENDPROC       _SETCOMMAND
  -------         PROC          _SETPAGE
  D:0007H         SYMBOL        p
  C:0533H         LINE#         54
  C:0533H         LINE#         55
  C:0533H         LINE#         56
  -------         ENDPROC       _SETPAGE
  -------         PROC          _SETLINE
  D:0007H         SYMBOL        p
  C:053AH         LINE#         59
  C:053AH         LINE#         60
  C:053AH         LINE#         61
  -------         ENDPROC       _SETLINE
  -------         PROC          _SETY
  D:0007H         SYMBOL        p
  C:0541H         LINE#         64
  C:0541H         LINE#         65
BL51 BANKED LINKER/LOCATER V6.22.2.0                                                  05/05/2022  21:30:59  PAGE 5


  C:0541H         LINE#         66
  -------         ENDPROC       _SETY
  -------         PROC          _NAME
  D:0006H         SYMBOL        line
  -------         DO            
  X:0064H         SYMBOL        l
  X:0065H         SYMBOL        j
  -------         ENDDO         
  C:0003H         LINE#         69
  C:0003H         LINE#         70
  C:0003H         LINE#         71
  C:000BH         LINE#         74
  C:002AH         LINE#         75
  C:002AH         LINE#         76
  C:0033H         LINE#         77
  C:0033H         LINE#         78
  C:0035H         LINE#         79
  C:0037H         LINE#         80
  C:0039H         LINE#         81
  C:003BH         LINE#         82
  C:003EH         LINE#         83
  C:0041H         LINE#         84
  C:004AH         LINE#         85
  C:004DH         LINE#         87
  C:004DH         LINE#         88
  C:004DH         LINE#         89
  C:004DH         LINE#         90
  C:0050H         LINE#         92
  C:0052H         LINE#         93
  C:0054H         LINE#         94
  C:0057H         LINE#         95
  C:005AH         LINE#         96
  C:0061H         LINE#         97
  C:0061H         LINE#         99
  C:0061H         LINE#         100
  C:0061H         LINE#         101
  C:0061H         LINE#         102
  C:0061H         LINE#         103
  C:0064H         LINE#         104
  C:0073H         LINE#         105
  C:0073H         LINE#         106
  C:0075H         LINE#         107
  C:0077H         LINE#         108
  C:0079H         LINE#         109
  C:007BH         LINE#         110
  C:007EH         LINE#         111
  C:0081H         LINE#         112
  C:0089H         LINE#         113
  C:008CH         LINE#         115
  C:008CH         LINE#         116
  C:008CH         LINE#         117
  C:008CH         LINE#         118
  C:008FH         LINE#         120
  C:0091H         LINE#         121
  C:0093H         LINE#         122
  C:0096H         LINE#         123
  C:0099H         LINE#         124
BL51 BANKED LINKER/LOCATER V6.22.2.0                                                  05/05/2022  21:30:59  PAGE 6


  C:009FH         LINE#         125
  C:009FH         LINE#         127
  C:009FH         LINE#         128
  C:009FH         LINE#         129
  C:009FH         LINE#         130
  C:009FH         LINE#         132
  C:00A1H         LINE#         134
  C:00A1H         LINE#         135
  C:00A3H         LINE#         136
  C:00A5H         LINE#         137
  C:00A7H         LINE#         138
  C:00A9H         LINE#         139
  C:00ACH         LINE#         140
  C:00AFH         LINE#         141
  C:00B8H         LINE#         142
  C:00BBH         LINE#         144
  C:00BBH         LINE#         145
  C:00BBH         LINE#         146
  C:00BBH         LINE#         147
  C:00BEH         LINE#         149
  C:00C0H         LINE#         150
  C:00C2H         LINE#         151
  C:00C5H         LINE#         152
  C:00C8H         LINE#         153
  C:00D1H         LINE#         154
  C:00D4H         LINE#         156
  C:00D6H         LINE#         157
  C:00D8H         LINE#         158
  C:00F2H         LINE#         159
  C:00F5H         LINE#         160
  C:00F5H         LINE#         161
  C:0106H         LINE#         162
  -------         ENDPROC       _NAME
  -------         PROC          CLEAR
  -------         DO            
  X:0064H         SYMBOL        i
  X:0066H         SYMBOL        j
  -------         ENDDO         
  C:0107H         LINE#         164
  C:0107H         LINE#         165
  C:0107H         LINE#         167
  C:0109H         LINE#         168
  C:010BH         LINE#         169
  C:0122H         LINE#         170
  C:0122H         LINE#         171
  C:0124H         LINE#         172
  C:0126H         LINE#         173
  C:012BH         LINE#         174
  C:012EH         LINE#         175
  C:0131H         LINE#         176
  C:0134H         LINE#         178
  C:013BH         LINE#         179
  C:013BH         LINE#         180
  C:013DH         LINE#         181
  C:013FH         LINE#         182
  C:0142H         LINE#         183
  C:0145H         LINE#         184
BL51 BANKED LINKER/LOCATER V6.22.2.0                                                  05/05/2022  21:30:59  PAGE 7


  C:0162H         LINE#         185
  C:0172H         LINE#         186
  C:0174H         LINE#         187
  C:0176H         LINE#         188
  C:018DH         LINE#         189
  C:018DH         LINE#         190
  C:018FH         LINE#         191
  C:0191H         LINE#         192
  C:0196H         LINE#         193
  C:0199H         LINE#         194
  C:019CH         LINE#         195
  C:019FH         LINE#         197
  C:01A6H         LINE#         198
  C:01A6H         LINE#         199
  C:01A8H         LINE#         200
  C:01AAH         LINE#         201
  C:01ADH         LINE#         202
  C:01B0H         LINE#         203
  C:01CDH         LINE#         204
  C:01DDH         LINE#         205
  -------         ENDPROC       CLEAR
  -------         PROC          MINICLEAR
  -------         DO            
  X:0064H         SYMBOL        i
  X:0066H         SYMBOL        j
  -------         ENDDO         
  C:01DEH         LINE#         208
  C:01DEH         LINE#         209
  C:01DEH         LINE#         211
  C:01E0H         LINE#         212
  C:01E2H         LINE#         213
  C:01F9H         LINE#         214
  C:01F9H         LINE#         215
  C:01FBH         LINE#         216
  C:01FDH         LINE#         217
  C:0202H         LINE#         218
  C:0205H         LINE#         219
  C:0208H         LINE#         220
  C:020BH         LINE#         222
  C:0212H         LINE#         223
  C:0212H         LINE#         224
  C:0214H         LINE#         225
  C:0216H         LINE#         226
  C:0219H         LINE#         227
  C:021CH         LINE#         228
  C:0239H         LINE#         229
  C:0249H         LINE#         230
  C:024BH         LINE#         231
  C:024DH         LINE#         232
  C:0264H         LINE#         233
  C:0264H         LINE#         234
  C:0266H         LINE#         235
  C:0268H         LINE#         236
  C:026DH         LINE#         237
  C:0270H         LINE#         238
  C:0273H         LINE#         239
  C:0276H         LINE#         241
BL51 BANKED LINKER/LOCATER V6.22.2.0                                                  05/05/2022  21:30:59  PAGE 8


  C:027DH         LINE#         242
  C:027DH         LINE#         243
  C:027FH         LINE#         244
  C:0281H         LINE#         245
  C:0284H         LINE#         246
  C:0287H         LINE#         247
  C:02A4H         LINE#         248
  C:02B4H         LINE#         249
  -------         ENDPROC       MINICLEAR
  -------         PROC          INIT
  C:04FEH         LINE#         250
  C:04FEH         LINE#         251
  C:04FEH         LINE#         252
  C:0500H         LINE#         253
  C:0502H         LINE#         254
  C:0504H         LINE#         255
  C:0506H         LINE#         256
  C:0508H         LINE#         257
  C:050BH         LINE#         258
  C:050EH         LINE#         260
  C:0510H         LINE#         261
  C:0512H         LINE#         262
  C:0514H         LINE#         263
  C:0517H         LINE#         264
  -------         ENDPROC       INIT
  -------         PROC          TEST
  -------         DO            
  X:0060H         SYMBOL        i
  X:0062H         SYMBOL        j
  -------         ENDDO         
  C:02B5H         LINE#         267
  C:02B5H         LINE#         268
  C:02B5H         LINE#         270
  C:02B7H         LINE#         271
  C:02B9H         LINE#         272
  C:02D0H         LINE#         273
  C:02D0H         LINE#         274
  C:02D2H         LINE#         275
  C:02D4H         LINE#         276
  C:02D9H         LINE#         277
  C:02DCH         LINE#         278
  C:02DFH         LINE#         279
  C:02E2H         LINE#         281
  C:02E9H         LINE#         282
  C:02E9H         LINE#         283
  C:02EBH         LINE#         284
  C:02EDH         LINE#         285
  C:02F0H         LINE#         286
  C:02F3H         LINE#         287
  C:0310H         LINE#         288
  C:0320H         LINE#         289
  C:0322H         LINE#         290
  C:0324H         LINE#         291
  C:033BH         LINE#         292
  C:033BH         LINE#         293
  C:033DH         LINE#         294
  C:033FH         LINE#         295
BL51 BANKED LINKER/LOCATER V6.22.2.0                                                  05/05/2022  21:30:59  PAGE 9


  C:0344H         LINE#         296
  C:0347H         LINE#         297
  C:034AH         LINE#         298
  C:034DH         LINE#         300
  C:0354H         LINE#         301
  C:0354H         LINE#         302
  C:0356H         LINE#         303
  C:0358H         LINE#         304
  C:035BH         LINE#         305
  C:035EH         LINE#         306
  C:037BH         LINE#         307
  C:038BH         LINE#         308
  -------         ENDPROC       TEST
  -------         ENDMOD        DISPLAY

*** WARNING L16: UNCALLED SEGMENT, IGNORED FOR OVERLAY PROCESS
    SEGMENT: ?PR?DELAY100US?DELAY

*** WARNING L16: UNCALLED SEGMENT, IGNORED FOR OVERLAY PROCESS
    SEGMENT: ?PR?_WRITEDATA?DISPLAY

*** WARNING L16: UNCALLED SEGMENT, IGNORED FOR OVERLAY PROCESS
    SEGMENT: ?PR?_SETPAGE?DISPLAY

*** WARNING L16: UNCALLED SEGMENT, IGNORED FOR OVERLAY PROCESS
    SEGMENT: ?PR?_SETLINE?DISPLAY

*** WARNING L16: UNCALLED SEGMENT, IGNORED FOR OVERLAY PROCESS
    SEGMENT: ?PR?_SETY?DISPLAY

*** WARNING L16: UNCALLED SEGMENT, IGNORED FOR OVERLAY PROCESS
    SEGMENT: ?PR?TEST?DISPLAY

Program Size: data=9.0 xdata=106 code=1352
LINK/LOCATE RUN COMPLETE.  6 WARNING(S),  0 ERROR(S)
